:100000000C9417060C94F3280C9420290C943F06AA
:100010000C943F060C94BD0C0C943F060C943F06C8
:100020000C943F060C943F060C943F060C943F063C
:100030000C943F060C943F060C943F060C943F062C
:100040000C944D290C943F060C94072D0C94422DD2
:100050000C943F060C943F060C943F060C943F060C
:100060000C943F060C943F06501C571C571C501C08
:10007000571C571C571C571C571C571C571C571CE8
:10008000571C571C571C571C571CC51B571C571C6B
:10009000571C571C571C281B571C571C571C571CF8
:1000A000571C571C571C571C571C571C571C571CB8
:1000B000571C571C571CD11BD11BD11BD11BD11B4B
:1000C000D11BD11BD11BD11B571C571C571C571CB4
:1000D000571C571C2D1BD01BD01BD01BD01B571CD3
:1000E000E11BE91BF11BF91B011C091C111C191C4C
:1000F000231C2D1C371C411C741B341B571C571C04
:10010000571C571CC51B571C571C571C571C571CEA
:10011000571C571C571CCF1BCF1BCF1BCF1B571C6B
:10012000E11BE91BF11BF91B011C091C111C191C0B
:10013000231C2D1C371C411C741B341B571C571CC3
:10014000571C571CC51B881C881C881C881C881CB5
:10015000881C881C881C881C881C881C881C881C7F
:10016000A81DA81DA81DA81DA81DA81DCF1CD91C11
:10017000E31CED1C531D5D1D6B1D7C1D191E891E8E
:100180005A1E5F1E641E691E6E1E731E781E891E17
:10019000831E8F25A425B025B925C625EC25F42579
:1001A00017260426456E746572206D656E752E2EB9
:1001B0002E00546F67676C6564206D6963726F50C1
:1001C000504D00546F67676C656420696E76657288
:1001D0007465642050504D2100546F67676C6564EE
:1001E000205458206D7574696E672100546F6767DD
:1001F0006C65642074656C656D657472792100505E
:10020000726F746F636F6C206572726F72207769A2
:1002100074682052580054696D656F757420776852
:10022000656E20636F6E6E656374696E6720746FB0
:1002300020525800507265737320616E79206B658F
:100240007920746F2063616E63656C00436F6E6E1E
:10025000656374696E6720746F2052582C20706F2C
:100260007765722075702074686520525820287751
:100270006974682062696E6420706C7567206966B5
:10028000206E6F74207573696E6720616C77617979
:10029000732062696E642900546F67676C6564201F
:1002A00027696D6D656469617465206F757470751B
:1002B000742700546F67676C65642027736C6176E0
:1002C00065206D6F64652700546F67676C656420F7
:1002D00027616C776179732062696E642700546FBF
:1002E00067676C65642050504D206368616E6E6571
:1002F0006C206C696D6974005365742052535349C6
:1003000020696E6A656374696F6E206368616E6EE2
:10031000656C2028303D3D64697361626C6529001D
:100320005365742050504D206D696E696D756D2058
:1003300073796E630053657420626561636F6E202C
:10034000696E74657276616C0053657420626561D4
:10035000636F6E2064656C6179005365742062651B
:1003600061636F6E206672657175656E6379206971
:100370006E20487A3A20303D64697361626C652C66
:100380002050783D504D52206368616E6E656C2040
:10039000782C2046783D465253206368616E6E6526
:1003A0006C2078005365742050574D2073746F7023
:1003B0002064656C61792028302064697361626C07
:1003C00065642C20312D323535203D3D20302E31D5
:1003D00073202D2035306D696E29005365742050CF
:1003E000504D2073746F702064656C6179202830E3
:1003F0002064697361626C65642C20312D3235355F
:10040000203D3D20302E3173202D2035306D696E1A
:100410002900536574206661696C736166652064A8
:10042000656C61792028302064697361626C656451
:100430002C20312D323535203D3D20302E3173209A
:100440002D2035306D696E29002A2A2A2A2A2A2A67
:100450002A2A2A2A2A2A2A2A2A2A2A2A2A2A2A2AFC
:100460002A2A2A2A2A2A0052582041636B656420CE
:100470002D2072657665727420737563636573737E
:1004800066756C21002A2A2A2A2A2A2A2A2A2A2A36
:100490002A2A2A2A2A2A2A2A2A2A2A2A2A2A2A2ABC
:1004A0002A2A002A2A2A2A2A2A2A2A2A2A2A2A2AD6
:1004B0002A2A2A2A2A2A2A2A2A2A2A2A2A2A2A2A9C
:1004C0000052582041636B6564202D207570646173
:1004D0007465207375636365737366756C21002A98
:1004E0002A2A2A2A2A2A2A2A2A2A2A2A2A2A2A2A6C
:1004F0002A2A2A2A2A2A2A2A2A2A2A2A0056616CE1
:1005000069642063686F69636573206172653A206E
:100510005B315D2D5B31365D20286368616E6E65F1
:100520006C20312D31362900536574206F7574703D
:10053000757420666F7220706F727420005B585D56
:100540002061626F7274206368616E6765732061F9
:100550006E64206578697420525820636F6E6669F6
:1005600067005B535D207361766520736574746901
:100570006E677320746F205258005B525D20726565
:10058000766572742052582073657474696E67734F
:1005900020746F2064656661756C747300557365B3
:1005A000206E756D62657273205B312D445D207421
:1005B0006F206564697420706F727473205B452DC1
:1005C000515D20666F722073657474696E67730085
:1005D000202D20726563656976657220636F6E6693
:1005E0006967757261746F722C207278207377203E
:1005F000000A0A6F70656E4C52536E672000536597
:10060000742073657269616C2062617564726174D3
:10061000653A200056616C69642063686F696365A0
:10062000733A2031202D20342B34202F2032202DDE
:100630002038202F2033202D20382B34202F203419
:10064000202D203132202F2035202D2031322B3407
:10065000202F2036202D203136005365742043682A
:10066000616E6E656C20636F6E6669673A20005339
:1006700065742044617461726174652028302D3284
:10068000293A200053657420486F70206368616EBA
:100690006E656C7320286D61782032342C20736570
:1006A0007061726174656420627920636F6D6D6141
:1006B00073292076616C69642076616C756573209E
:1006C000312D3235353A2000536574206368616EF0
:1006D0006E656C2073706163696E672028783130B5
:1006E0006B487A293A200053657420524620706F77
:1006F0007765722028302D37293A20005365742001
:100700005246206D616769632028686578292065F5
:100710002E672E20307844454144463030443A20FC
:10072000005365742062617365206672657175653A
:100730006E63792028696E20487A293A20005B5A36
:100740005D20656E74657220726563656976657299
:1007500020636F6E66696775726174696F6E20756C
:1007600074696C79005B465D20646973706C6179B3
:100770002061637475616C206672657175656E6366
:100780006965732075736564005B525D2063616CFD
:1007900063756C6174652072616E646F6D206B654A
:1007A0007920616E6420686F70206C697374005BDF
:1007B000495D207265696E697469616C697A65204A
:1007C00073657474696E677320746F20736B6574DE
:1007D00063682064656661756C7473005B585D20A6
:1007E000726576657274206368616E6765732061F7
:1007F0006E642065786974206D656E75005B535D6D
:1008000020736176652073657474696E67732074F4
:100810006F20454550524F4D20616E6420657869C8
:1008200074206D656E7500557365206E756D62651B
:100830007273205B302D395D20746F20656469749C
:1008400020706172616D657465727300202D205394
:10085000797374656D20636F6E6669677572617414
:10086000696F6E000A0A6F70656E4C52536E672096
:10087000005129204F7574707574206265666F721F
:1008800065206C696E6B20283D465329203A200074
:10089000502920536C617665206D6F646520286552
:1008A00078706572696D656E74616C293A20004FCD
:1008B000292054696D65642042494E4420617420AA
:1008C0007374617274757020203A20004E29205094
:1008D000504D206F7574707574206C696D69746506
:1008E0006420202020203A200044495341424C45B6
:1008F00044004D292050504D205253534920746FCD
:10090000206368616E6E656C202020203A20004CC8
:10091000292050504D206D696E696D756D20737979
:100920006E63202875732920203A200044495341E2
:10093000424C4544004B29204661696C73616665F1
:1009400020626561636F6E20696E74762E20283197
:100950002D32353573293A20004A29204661696CC9
:100960007361666520626561636F6E2064656C61AA
:10097000792028302D323535203D3E20313073200E
:100980002D203135306D696E293A200049292046E5
:1009900061696C7361666520626561636F6E206674
:1009A00072712E203A200048292050574D20737430
:1009B0006F702064656C6179202020202020203A0F
:1009C000200047292050504D2073746F70206465BB
:1009D0006C6179202020202020203A200046292008
:1009E0004661696C736166652064656C617920207D
:1009F00020202020203A200050574D206368616E4F
:100A00006E656C200066756E6374696F6E3A2000C7
:100A10002920706F72742000506F776572546F7761
:100A2000657200445446205548462033322D626991
:100A3000742031306368004F70656E4C52536E679E
:100A40005258206D696E6920342F36636800466CF9
:100A50007974726F6E2F4F72616E676552582055B0
:100A600048462038636800525820747970653A20EF
:100A70000044697361626C656400487A00203D3D02
:100A8000200043616C63756C617465642070616300
:100A90006B657420696E74657276616C3A200042F1
:100AA00029204D6963726F202868616C6629205087
:100AB000504D202020203A00412920496E76657251
:100AC0007465642050504D20696E20202020203A0B
:100AD000003029204D7574652062757A7A65722020
:100AE000286D6F73746C79293A0039292053657227
:100AF00069616C2062617564726174653A00736D3E
:100B0000617274506F7274004672536B7900547244
:100B1000616E73706172656E740044697361626CBA
:100B200065640038292054656C656D657472793A86
:100B300020202020202020003729204368616E6E6D
:100B4000656C20636F6E6669673A20200036292045
:100B500044617461726174652028302D32293A2015
:100B6000202000352920486F70206368616E6E6513
:100B70006C733A2020202020003429204368616EC5
:100B80006E656C2073706163696E673A2020003374
:100B90002920524620706F7765722028302D372922
:100BA0003A202020003229205246206D6167696377
:100BB0003A202020202020202020003129204261BE
:100BC0007365206672657175656E63793A202020C1
:100BD0000000000000240027002A0000000000257B
:100BE0000028002B0000000000230026002900043C
:100BF00004040404040404020202020202030303C4
:100C000003030301020408102040800102040810BD
:100C1000200102040810200000000700020100006B
:100C2000030406000000000000000000EA2E11246A
:100C30001FBECFEFD8E0DEBFCDBF13E0A0E0B1E034
:100C4000E6E1F0E602C005900D92A839B107D9F7A8
:100C500016E0A8E9B3E001C01D92A935B107E1F79C
:100C60001CE0CEE2DCE004C02297FE010E94E62FE9
:100C7000CC32D107C9F70E942F2F0C9409300C9465
:100C80000000A0E0B0E0E7E4F6E00C94B52FEC0142
:100C9000A880B980CA80DB80A114B104C104D1044A
:100CA00041F484E2A82E89EDB82E8BE5C82E87E0AA
:100CB000D82EC601B5012DE133EF41E050E00E948E
:100CC000922F27EA31E440E050E00E943E2F7B0162
:100CD0008C01C601B5012DE133EF41E050E00E94E7
:100CE000922FCA01B9012CEE34EF4FEF5FEF0E9453
:100CF0003E2F6E0D7F1D801F911F97FF04C0615016
:100D0000704080409048688379838A839B839B01ED
:100D1000AC015F77B901CA01CDB7DEB7EAE00C9448
:100D2000D12F0E944106089581EB92E00E94410676
:100D300008956093B1027093B2028093B3029093CE
:100D4000B4020895A0E0B0E0E8EAF6E00C94AE2F1B
:100D5000EC012B016A016115710519F0FB0191830A
:100D60008083C114D10449F0C6010297839728F00B
:100D700020E030E040E050E0DCC0A9908A2D90E017
:100D80000E94FE2F892BC9F7FDE2AF1621F4A9902E
:100D90003324339405C08BE2A81609F4A9903324B8
:100DA000C114D10421F0E0E1CE16D10411F5F0E335
:100DB000AF1669F48881883711F0883541F4A9802D
:100DC000229682E0382A20E1C22ED12C12C0C11412
:100DD000D10479F4E0E3AE1659F199E9E92E99E9E5
:100DE000F92E99E9092F99E1192F8AE0C82ED12C03
:100DF0003AC0FAE0CF16D10491F080E1C816D104D0
:100E000029F0E8E0CE16D104F9F415C0BFEFEB2EBF
:100E1000BFEFFB2EBFEF0B2FBFE01B2F24C0A9E9B4
:100E2000EA2EA9E9FA2EA9E90A2FA9E11A2F1BC077
:100E3000F8E0CF2ED12CEFEFEE2EEFEFFE2EEFEFFE
:100E40000E2FEFE11E2F0FC09601442737FD40956E
:100E5000542F6FEF7FEF8FEF9FEF0E94702FC9012C
:100E6000DA017C018D0120E030E040E050E060E0FC
:100E70003601882477FC8094982C70EDB72EBA0C3C
:100E8000F9E0FB1570F48A2D81548A3118F499EC3D
:100E9000B92E06C08A2D81568A3148F589EAB82EC6
:100EA000BA0C8B2D90E08C159D050CF56F3FE9F089
:100EB000E216F30604071507B8F0CA01B901A40148
:100EC00093010E943E2F9B01AC018B2D90E0A0E08E
:100ED000B0E0280F391F4A1F5B1F281739074A0740
:100EE0005B0710F061E001C06FEFA990C6CF41141D
:100EF000510451F0662311F0219703C031FE04C064
:100F00002297F201D183C08330FE07C050954095EF
:100F1000309521953F4F4F4F5F4F67FF0AC082E2E8
:100F200090E090935806809357062FEF3FEF4FEFD6
:100F30005FEFB901CA01CDB7DEB7E1E10C94CA2F6A
:100F4000FC0188279927E89421912032E9F3293080
:100F500010F02E30C8F32B3241F02D3239F4689462
:100F600004C00E94F507820F911D219120532A3061
:100F7000C0F31EF4909581959F4F089548E953E082
:100F80000E94C3070895009731F4DA018D919C9176
:100F9000009709F40EC0DC01FB013D912191222351
:100FA00019F03217C9F3FACF332331F4DA011D9265
:100FB0001C928827992708951197AF93BF93FB013F
:100FC0003D912191321771F4332321F48827992719
:100FD000119702C01E921196FA01A193B0839F91BE
:100FE0008F910895222369F7EACF7AE0979F902D99
:100FF000879F802D910D1124089580919A0381304F
:1010000019F482E080939A0380919A03833019F453
:1010100084E080939A030895E3E0F0E089E0809310
:101020005700849190E08670863009F491E0892F12
:1010300008951F93182F0E940C08882379F09FB7FA
:1010400081E080939F05F894A89588E180936000E3
:1010500010936000112309F0A8959FBF1F91089578
:10106000382F20E080913105909132058227932717
:1010700040E061E270E19C01220F331F97FF04C042
:10108000C9018627972701C0C9014F5F483099F7EA
:101090009093320580933105089587E38093D003C0
:1010A00080E092ECA1E0B0E08093D1039093D20372
:1010B000A093D303B093D40387E08093DD0380E053
:1010C00091EAACEBB3E38093D5039093D603A0935E
:1010D000D703B093D80385E08093DE038DEE9EEFB7
:1010E000ADEABEED8093D9039093DA03A093DB03BE
:1010F000B093DC03AFEDB3E080E090E0863010F019
:10110000E0E004C0FC01EF57FC4FE081ED93019655
:101110008831910599F782E08093F7038AE0809304
:10112000F803089580E09EECADEEB4E380939D0358
:1011300090939E03A0939F03B093A00380E090E060
:10114000A0E0B0E58093A1039093A203A093A30332
:10115000B093A403E5EAF3E080E081938F5F8031F0
:10116000E1F708958436910520F4BC0180E090E019
:1011700025C08E3B910550F48A559040BC0180E01B
:1011800090E02AE030E040E050E016C0823D91055A
:1011900050F4845B9040BC0180E090E024E630E0B5
:1011A00040E050E009C08D5C9040BC0180E090E0E0
:1011B00028E532E040E050E00E943E2F24E630E097
:1011C00040E050E00E943E2F089590E08C599F4FE0
:1011D0000E94B2080895DC019896EC91F0E0E77067
:1011E000F070E758FC4F808108958F929F92AF92E4
:1011F000BF92CF92DF92EF92FF920F931F938C01D9
:101200000E94EB08D80197962C9130E043E150E022
:10121000249FF001259FF00D349FF00D1124EB5415
:10122000FD4F80809180A280B38090E00F96AA2726
:1012300097FDA095BA2FBC01CD0120E43FE14DE719
:1012400050E00E943E2FA50194010E94702F690179
:101250007A0180ED97E0A0E0B0E0C80ED91EEA1E4A
:10126000FB1ED80198968C91887181F060E07EEE2B
:101270008AEB9BE0A50194010E94702F28513C4FFE
:101280004F4F5F4FC20ED31EE41EF51E87EE93E054
:10129000A0E0B0E0C80ED91EEA1EFB1EC701B601D1
:1012A00028EE33E040E050E00E94702FCA01B901FF
:1012B00028EE33E040E050E00E943E2F1F910F9156
:1012C000FF90EF90DF90CF90BF90AF909F908F9066
:1012D00008958F3F910509F010F480E0089522E011
:1012E0008030920710F481E008958050934010F010
:1012F00083E0089582E00895CF92DF92FF920F93EA
:101300001F93CF93DF93F82FEB016A01182F1695E7
:10131000E0E088819981D6018C938A819B81119626
:101320008C9311978C819D8112968C9312978E814C
:101330009F8113968C931397288139814A815B8111
:101340006C817D818E819F819295990F990F907C00
:10135000832F8370982B852F8370880F880F982B8D
:10136000872F83708295807F982B14969C9385E0BD
:1013700090E0C80ED91E2896EF5F1E1750F6F0FFBA
:1013800021C0888199810E946909F82E8A819B81F8
:101390000E946909182F8C819D810E946909082F7C
:1013A0008E819F810E946909F294FF0CFF0C70EC02
:1013B000F7221295107F1F29182B000F000F012B09
:1013C000D6010C93DF91CF911F910F91FF90DF9089
:1013D000CF90089523E08032920718F420E030E0A7
:1013E00026C023E0883E920748F49C012F513340E9
:1013F00054E0369527955A95E1F719C027E0803DCE
:10140000920720F49C012C5D334011C028E08839FC
:10141000920718F02FEF33E00AC09C01285C374098
:1014200044E0369527954A95E1F72D503C4FC90188
:1014300008958C30910548F49C0174E0220F331F0D
:101440007A95E1F7285D3C4F17C023E0843F92076F
:1014500020F49C0124523C4F0FC024E080309207BE
:1014600018F020E938E008C09C012657334F64E0AB
:10147000220F331F6A95E1F7C90108959C01369543
:10148000279525753575821B930B9C0136952795FD
:10149000369527952373337383739373280F391FFE
:1014A000C901E4E096958795EA95E1F7820F931FCD
:1014B0008F709F7021E031E0AC01429FC001439FDB
:1014C000900D529F900D1124892F0895882339F093
:1014D0005F980000289A00005F9A000008955F98C6
:1014E0000000289800005F9A000008955F9A0000AD
:1014F00083B15F98000090E096958795817008957C
:101500000F931F93082F5C9A5F985C9810E0802FD0
:1015100080780E94660A000F1F5F1830C1F75F983D
:101520001F910F9108958F770E94800A08950F935D
:101530001F93082F10E0802F80780E94660A000F0A
:101540001F5F1830C1F75F981F910F9108950F9397
:101550001F935F9880E000E0182F110F0E94760A19
:10156000810F0F5F0830C1F71F910F9108950E94FE
:10157000930A0E94A70A5C9A08951F93162F806809
:101580000E94800A812F0E94970A5C9A1F910895F9
:101590001F931091D9031827E0EDF3E0E80FF11D38
:1015A00089E767850E94BD0A8DE3612F0E94BD0A0D
:1015B00082E4612F0E94BD0A1F91089586E20E9475
:1015C000B70A08950F931F938C018CE1F801648191
:1015D0000E94BD0A8DE1F80165810E94BD0A8EE17D
:1015E000F80166810E94BD0A80E2F80167810E94CD
:1015F000BD0A81E2F80160850E94BD0A82E2F8011D
:1016000061850E94BD0A83E2F80162850E94BD0ADD
:1016100084E2F80163850E94BD0A85E2F8016485D1
:101620000E94BD0A8AE2F80165850E94BD0A8EE625
:10163000F80166850E94BD0A8FE6F80167850E9461
:10164000BD0A80E7F80160890E94BD0A81E7F801C0
:1016500061890E94BD0A82E7F80162890E94BD0A81
:101660001F910F910895EF92FF920F931F93CF93C5
:10167000DF937B018C01603028E372072CE982073D
:101680002CE1920728F520E836E948E950E00E946D
:10169000702FE9016897B90180E090E020E839E611
:1016A00047E65FEF0E943E2F6E0D7F1D801F911F4A
:1016B00032E0660F771F881F991F3A95D1F721E70F
:1016C00032E040E050E00E94702F890180E421C0A8
:1016D00020E03DE241E351E00E94702FE90168976C
:1016E000B90180E090E020E033ED4EEC5EEF0E9427
:1016F0003E2F6E0D7F1D801F911F660F771F881F65
:10170000991F21E732E040E050E00E94702F8901EC
:1017100080E69E012F71622F680F85E70E94BD0A47
:1017200086E7612F0E94BD0A87E7602F0E94BD0AED
:10173000CDB7DEB7E6E00C94D52F9F92AF92BF9263
:10174000CF92DF920F93DF93CF9300D000D0CDB72D
:10175000DEB7982E83E00E94B70A8093F90384E0F5
:101760000E94B70A8093FA0386E060E00E94BD0AF7
:1017700087E061E00E94BD0A89E06FE70E94BD0A30
:101780008AE065E00E94BD0A8BE062E10E94BD0A2A
:101790008CE065E10E94BD0A8DE06DEF0E94BD0AFC
:1017A0008EE060E00E94BD0A992019F084E193E088
:1017B00008C08091F70323E1829FC00111248B545C
:1017C0009D4F0E94E20A80E36CE80E94BD0A82E31A
:1017D0006FE00E94BD0A83E362E40E94BD0A84E3D5
:1017E0006AE00E94BD0A85E36AE20E94BD0A86E3C0
:1017F0006DE20E94BD0A87E364ED0E94BD0A88E3A2
:1018000060E00E94BD0A89E360E00E94BD0A992061
:1018100049F065E8A62E61ECB62E61ECC62E6EEDA1
:10182000D62E08C0A090D903B090DA03C090DB0395
:10183000D090DC030AE38D2D9927AA27BB27898343
:101840009A83AB83BC83802F69810E94BD0A802F5D
:101850008B5F69810E94BD0ADC2CCB2CBA2CAA2498
:101860000F5F0E3341F783E46FEF0E94BD0A84E4FB
:101870006FEF0E94BD0A85E46FEF0E94BD0A86E407
:101880006FEF0E94BD0A992019F08DE666E003C053
:101890008DE66091DD030E94BD0A89E760E00E9449
:1018A000BD0A8AE76091DE030E94BD0A83E760E01B
:1018B0000E94BD0A84E760E00E94BD0A992029F0D9
:1018C00060E071EA8CEB93E308C06091D5037091FE
:1018D000D6038091D7039091D8030E94330B0F90C9
:1018E0000F900F900F90CF91DF910F91DF90CF90DD
:1018F000BF90AF909F90089587E061E00E94BD0A7D
:101900008EE764E20E94BD0A88E063E00E94BD0A9F
:1019100088E060E00E94BD0A87E065E00E94BD0AA1
:1019200085E062E00E94BD0A83E00E94B70A8093CE
:10193000F90384E00E94B70A8093FA030895582FB0
:1019400040919E04842F90E0FC01EF70F0709F01A5
:101950002F5F3F4F74E0959587957A95E1F72817AB
:10196000390751F0E257FB4F5083842F8F5F8F7000
:10197000407F842B80939E0408951F920F920FB690
:101980000F921124EF92FF920F931F932F933F9387
:101990004F935F936F937F938F939F93AF93BF9377
:1019A000EF93FF93E090A103F090A2030091A303B3
:1019B0001091A40389B1A801970120743070407080
:1019C000507090E063E0969587956A95E1F7A0E006
:1019D000B0E081709070A070B070281739074A0786
:1019E0005B0709F46AC02091840030918500109251
:1019F0008500109284008091BF04882309F05DC0A7
:101A0000E5FC02C03695279589E0253C3807C8F1EA
:101A100080914703A80197011CE15695479537959A
:101A200027951A95D1F7211531054105510521F466
:101A300021E030E040E050E090E0A0E0B0E0281786
:101A400039074A075B07D0F4809147038F3FB1F015
:101A500020E00EC0E22FF0E0EE0FFF1FDF01A054E8
:101A6000BB4F8D919C91E95DFC4F918380832F5FEB
:101A700080914703281770F31092BE041092470319
:101A80001CC082E02D3B3807A8F0809147038031CD
:101A900088F410914703C9010E94EA09E12FF0E0A0
:101AA000EE0FFF1FE054FB4F918380831F5F109365
:101AB000470303C08FEF80934703FF91EF91BF91DE
:101AC000AF919F918F917F916F915F914F913F91D6
:101AD0002F911F910F91FF90EF900F900FBE0F90DD
:101AE0001F90189583E0809380008AE180938100A5
:101AF0008FEF9FEF909389008093880010926F0082
:101B000088E080936D00E8E6F0E080818460808367
:101B100008956F3018F086958058089589E0689F81
:101B2000802D11240895882319F460E071E002C02B
:101B300063E071E085E396E00E94F22C0895A0E056
:101B4000B0E0E5EAFDE00C94B72F182F0E94A3291E
:101B50009B01AC0180912B0590912C05A0912D0546
:101B6000B0912E0569017A01C81AD90AEA0AFB0A5E
:101B7000D701C60189589341A040B04010F010929F
:101B80002A0520932B0530932C0540932D05509367
:101B90002E052091BF04822F81508230E8F580917C
:101BA0002A05882309F44FC1813011F482E0BCC1B9
:101BB000803108F035C1E82FF0E0E054FB4F10838E
:101BC0008F5F80932A05803109F0B0C1A2ECB4E0A8
:101BD000213039F41196EC911197E695E6958C91A8
:101BE00009C08D919C911197E92FE695E695E695B0
:101BF00096958795E03140F4F0E090E0EE0FFF1FFE
:101C0000E95DFC4F918380831092BE04129684E0BC
:101C1000A03DB807E9F68AC1233009F004C18091DC
:101C20002A05882321F41F3009F080C10CC18831B6
:101C300030F4E82FF0E0E154FB4F108374C1883199
:101C400009F0EEC0112309F0EBC0C0E0D0E00BE0DA
:101C500010E0DE0163E0AA0FBB1F6A95E1F7C09FA9
:101C6000B001C19F700DD09F700D1124FB01E05495
:101C7000FB4F80812181922F977095958795FD016B
:101C8000EE0FFF1FE95DFC4F91838083FB01EF5353
:101C9000FB4F30813695369536952181422F4295FE
:101CA000440F407E842F832B269526952695922FD0
:101CB000977095958795FD01EE0FFF1FE75DFC4F2F
:101CC00091838083FB01EE53FB4F80818295869543
:101CD000869583704181942F990F990F292F282B76
:101CE000429546954695437082818170880F880F92
:101CF000382F342B35952795FD01EE0FFF1FE55D3D
:101D0000FC4F31832083FB01EC53FB4F3081369530
:101D10002181422F479544274795842F832B269571
:101D2000922F977095958795FD01EE0FFF1FE35D4C
:101D3000FC4F91838083FB01EB53FB4F3081329545
:101D40003F702181422F4295407F842F832B229523
:101D50002F70922F977095958795FD01EE0FFF1FBD
:101D6000E15DFC4F91838083FB01EA53FB4F80814F
:101D7000881F8827881F4181942F990F292F282B8E
:101D8000441F4427441F82818370880F382F342BCF
:101D900035952795FD01EE0FFF1FEF5CFC4F31835A
:101DA0002083FB01E853FB4F308136953695218126
:101DB000422F4295440F440F407C842F832B26955D
:101DC0002695922F977095958795AA0FBB1FFD01B9
:101DD000ED5CFC4F9183808367537B4FFB01208137
:101DE0002295269527704181342F330F330F330FFF
:101DF000832F822B942F9295969597709595879522
:101E0000AB5CBC4F11969C938E932196C230D1054A
:101E100009F01FCF8091D60483FD02C01092BE044A
:101E200010922A0583C0243009F080C040912A0511
:101E3000442359F4183AB1F4109232051092310546
:101E400088EA0E94300881E06FC0413019F4109395
:101E50002F0504C0423031F410933005812F0E94C9
:101E600030085DC060913005262F30E0220F331F0F
:101E7000E42FF0E0C90102968E179F0734F0433239
:101E800068F7E354FB4F1083E9CF2D5F3F4F40913C
:101E9000310550913205E217F30749F4912F80E0A4
:101EA00048275927509332054093310538C0812F78
:101EB00090E04817590789F580912F05813069F521
:101EC000613118F080E180933005D0903005F0EC5E
:101ED000EF2EF4E0FF2E00E010E01BC0F701D081F0
:101EE000C0E0818190E08C2B9D2BE3E09695879557
:101EF000EA95E1F70E94EA09F801EE0FFF1FE95D9C
:101F0000FC4F918380830F5F1F4F82E090E0E80ECB
:101F1000F91E0D1518F31092BE0410922A05809137
:101F20002A05882319F08F5F80932A05CDB7DEB785
:101F3000E8E00C94D32FFF920F931F93CF93DF937E
:101F4000182F092FF62E8EE30E94BD0A212F302F65
:101F5000C901EC0110E005C08FE769910E94BD0A3C
:101F60001F5F1F15C8F385E064E00E94BD0A83E08F
:101F70000E94B70A8093F90384E00E94B70A809315
:101F8000FA030E94A3296093FB037093FC038093E0
:101F9000FD039093FE0387E069E00E94BD0A81E0A3
:101FA00080939A03CDB7DEB7E5E00C94D62F0E945C
:101FB0009B0F80919A038130D9F40E94A32920912C
:101FC000FB033091FC034091FD035091FE03621B23
:101FD000730B840B950B605A76488140904040F417
:101FE000E8CF85E396E067E071E00E94F22C089567
:101FF00080919A038130A9F3089585E396E06EE716
:102000000E94AA2E0895A0E0B0E0E9E0F0E10C946F
:10201000B62F6C0185E396E06EE70E94AA2E76014A
:1020200000E010E0C0E0D0E0B0E2BB2E0AC0083013
:10203000110521F49E012095F60120870894E11CEA
:10204000F11CF7016081862F8D57823040F485E3C3
:1020500096E06DE70E94AA2EF70160816B2585E36B
:1020600096E00E94AA2E0115110551F0F70180811A
:102070009E01280F311DC32FDD27C20FD31FD07043
:102080000F5F1F4F0930110591F6CDB7DEB7E9E0BC
:102090000C94D22FA9E0B0E0E0E5F0E10C94BD2F64
:1020A000382FE62F8091A30490E0019664E270E05F
:1020B0000E945D2F982F8093A30488E9898380E193
:1020C0008A83913071F0913028F0923099F09330FA
:1020D000E1F416C085E08B8381EF8C832F5F2D8325
:1020E00017C09B8381EF8C8384E6489FC001112435
:1020F0009D830EC084E08B8381EF8C833D8308C079
:102100009B8381EF8C83ED8303C00E94FD0F04C08D
:10211000CE0101960E9403102996E2E00C94D92F7B
:102120000F931F93CF93DF93182F092F85E396E02A
:102130006EE70E94AA2E212F302FC901EC0110E07A
:1021400000E288818D57823040F485E396E06DE7A8
:102150000E94AA2E88818027888385E396E0699172
:102160000E94AA2E1F5F193061F785E396E06EE7A3
:102170000E94AA2EDF91CF911F910F910895A9E09F
:10218000B0E0E5ECF0E10C94BD2F382F8091A30472
:10219000882379F48EEF89833A836B83842F90E0D0
:1021A000959587958C832D83198618861F821E82AC
:1021B0002FC040919E04842F90E09C012F703070BE
:1021C00054E0959587955A95E1F78217930721F189
:1021D0008DEF89831A821B82DE01149620E008C0ED
:1021E000E257FB4F80818D93405F2F5F263069F06F
:1021F000842F90E0FC0134E0F595E7953A95E1F7FE
:102200008F709070E817F90759F740939E042A835E
:10221000CE0101960E9490108091A30490E0019657
:1022200066E070E00E945D2F8093A3042996E2E0AF
:102230000C94D92F9F92AF92BF92CF92DF92EF92E0
:10224000FF920F931F93B82EA62ED42EC22E902E3F
:102250000E94A3297B018C0180918D0420919F0411
:102260003091A0044091A1045091A2048823B1F0C0
:10227000D801C701821B930BA40BB50B815E9E4254
:10228000A040B04020F12C2DDC1408F42D2D8B2D16
:102290006A2D422F292D0E944A1011C0D801C70172
:1022A000821B930BA40BB50B81539547A040B04004
:1022B00070F08B2D6A2D4D2D2C2D0E94BF10E092B9
:1022C0009F04F092A0040093A1041093A2041F9114
:1022D0000F91FF90EF90DF90CF90BF90AF909F90C5
:1022E000089585E396E0609100040E94AA2E089567
:1022F0001F93182F85E396E0612F0E94AA2E8091EC
:1023000000048127809300041F9108951F93192FC3
:102310000E947811812F0E9478111F910895DF92F9
:10232000EF92FF920F931F93D82E7B01109200041F
:1023300005E316E0C80165EB0E94AA2EC80162E61B
:102340000E94AA2E8D2D0E947811C7010E9486112D
:102350001F910F91FF90EF90DF900895E82FF0E02C
:10236000E456FC4FE185E03148F4F0E0EE0FFF1F4A
:10237000E95DFC4F0190F081E02D0DC0E03129F0C6
:10238000E13129F0E0E0F2E006C082E101C083E142
:102390000E94F72AFC01CF01089589E060E00E94C5
:1023A000282A88E061E00E94282A87E061E00E94F4
:1023B000282A82E060E00E94282A84E061E00E94EE
:1023C000282A0895892B19F08AE061E002C08AE08A
:1023D00060E00E94942A0895A0E2B0E0E2EFF1E10B
:1023E0000C94B52F8CE00E94B70A882379F585E319
:1023F00096E063E171E00E94F22C2D9A80E00E9449
:102400009D0B0E947C0C2D9821C085E396E00E94D4
:10241000712E482F8091BF04882321F0842F0E94C1
:102420009F0D14C080912805E82FF0E031969F01A0
:102430002F71307031978091270590E02817390768
:1024400029F0E250FB4F40832093280585E396E076
:102450000E94372E892BC9F680919A03843009F0A7
:102460008EC00E94A3296093AE047093AF04809342
:10247000B0049093B104611571058105910561F473
:1024800081E090E0A0E0B0E08093AE049093AF04D0
:10249000A093B004B093B1048091BA049091BB04AE
:1024A00081609093BB048093BA0483E080939A0385
:1024B0008FE70E94930A05EF14E00E94A70AF80133
:1024C00081938F01F4E00E3F1F07B9F74091E004BC
:1024D0008091F504282F30E0842F90E08227932705
:1024E00086FF40C080E448274093E004C901887318
:1024F0009070C89709F510E014C01F5F8091F80331
:10250000E12FF0E084FF06C0EB50FB4F80810E947A
:102510009F0C07C0EB50FB4F85E396E060810E9463
:10252000AA2E212F30E08091F50490E08770907002
:102530008217930714F716C02F733070232B91F472
:102540008091F6048093B2048091F7048093B404E0
:102550008091F8048093B5048091FB048093BC04BF
:102560001092BD0480912905813019F482E0809396
:10257000290580912905833011F4109229050E94C4
:10258000A3295B016C018091B6049091B704A091DE
:10259000B804B091B9040097A105B105C9F086014E
:1025A0007501E81AF90A0A0B1B0BD801C701885BF1
:1025B0009B40A040B04060F00E94DE0A8093B304CC
:1025C0001092B6041092B7041092B8041092B90495
:1025D00080ED93E00E94F5082091AA043091AB04AD
:1025E0004091AC045091AD0486017501E21AF30AE2
:1025F000040B150BE616F7060807190708F40DC1BA
:10260000A092AA04B092AB04C092AC04D092AD04E4
:10261000A8958091BE048830A0F08091A10390918C
:10262000A203A091A303B091A403FCE1B695A795E2
:1026300097958795FA95D1F70097A105B10509F00F
:102640008BC18091BE048F5F8093BE04E090AE0486
:10265000F090AF040091B0041091B104E114F104C2
:102660000105110511F180ED93E00E94F508AE1807
:10267000BF08C00AD10A6A157B058C059D0588F440
:102680008091A10384FD04C080ED97E00E94E211D7
:102690001092AE041092AF041092B0041092B104E4
:1026A00004C080E090E00E94E2119091E004907CF0
:1026B0009093E00400912805109127050117B1F1CE
:1026C00080912905823091F590589093E00480ED37
:1026D00093E00E94EB08893010F048E002C0482FD8
:1026E000415030E013C03F5FA32FB0E0812F90E056
:1026F000FC01E250FB4F2081FD01E052FB4F2083A3
:10270000A25EBA4F2C930196182F1F71341710F444
:10271000101749F710932705832F895C9091E004E7
:10272000892B8093E00430931E051AC0209129055F
:102730002430D1F490911E05EFE1F5E0A1EEB4E074
:10274000292F30E02E0F3F1F02C081918D93E21799
:10275000F307D9F7995C8091E004982B9093E004FB
:1027600083E08093290537C08091A504823029F445
:1027700091609093E0042D9A0FC09093E0042D98FF
:10278000222319F481E08093290580912905833063
:1027900019F484E080932905F89405EA13E07E019A
:1027A0000894E11CF11CF80181918F010E94AE1187
:1027B000F701819391937F01F3E0053B1F0799F7A0
:1027C0008091F8038770BE016F5F7F4F41EE54E048
:1027D0000E947C0978942C9A8091A4040E94C80AD3
:1027E00080ED93E00E94EB08682F80EE94E00E9459
:1027F0009B0FE091A404EF5FE093A404E83131F073
:10280000F0E0E053FC4F8785882339F41092A4044C
:1028100004C02D9A89E08093BE048091F8038871EA
:1028200071F180919A03823051F58091BA049091B0
:10283000BB04880F991F9093BB048093BA0483E074
:1028400080939A030E947C0C0E94A3296093B60493
:102850007093B7048093B8049093B904611571051F
:102860008105910561F481E090E0A0E0B0E0809303
:10287000B6049093B704A093B804B093B9048091C0
:10288000F80384FF1EC08091BA049091BB048E7F30
:102890000E943E0A182F8091B2046091BC040E94ED
:1028A000890D082F8091B304612F0E94890D282F74
:1028B0008091B4046091B504402F00919B030E9465
:1028C0001A112C988091A5048130D1F0813020F02C
:1028D000823009F047C034C08BE00E94C72A892BA0
:1028E00009F040C081E08093A5040E94952960937F
:1028F000A6047093A7048093A8049093A90432C0FF
:102900008BE00E94C72A892B21F50E9495292091EE
:10291000A6043091A7044091A8045091A904621B19
:10292000730B840B950B695E734080409040D0F030
:1029300082E08093A50480ED97E00E94E21112C02E
:102940008BE00E94C72A892B69F080E090E00E940A
:10295000E2111092A50406C08091BE04883009F0EF
:1029600059CF57CFA096EAE00C94D12F8AE061E0CE
:102970000E94282A8AE060E00E94942A08951F930A
:10298000182F0E94A32960939F047093A004809342
:10299000A1049093A20410938D04112329F440E81C
:1029A00055E260E070E004C040E051EE60E070E0AD
:1029B00085E396E00E94B02D1F910895ACE1B0E050
:1029C000E4EEF4E10C94B52F0E94A3297B018C0165
:1029D00081E00E949D0B84E7A82E6E010894C11C23
:1029E000D11CB3E0BB2EA982C60161E00E94D70FC3
:1029F000B0929A030E947C0C6AEF70E080E090E055
:102A00000E94C92980919A03833009F07DC085E333
:102A100096E00E94372E892B09F076C00E94A329E8
:102A20006E197F09800B910B6058734C894C914053
:102A300008F06AC0D8CF8FE70E94930A0E94A70AC5
:102A4000843509F05CC089830E94A70A182F00E032
:102A500010938C0400938B040E94A70A080F111D89
:102A600010938C0400938B040E94A70A80938A041D
:102A70000E94A70A80938904813108F040C0FF2496
:102A800007C00E94A70A07591B4FF8018083F394DF
:102A90000F2D10E08091890490E0880F991F08178E
:102AA000190778F380E78983CE01019661E00E94DF
:102AB000D70F83E080939A030E947C0C62E370E05E
:102AC00080E090E00E94C92980919A038330A9F0A8
:102AD0008FE70E94930A0E94A70A803581F48983B8
:102AE00005EB13E00E94A70AF80181938F01F3E040
:102AF000003D1F07B9F781E003C082E001C083E019
:102B00006C96EAE00C94D12F80919A03833009F0FF
:102B100092CFF3CF83E00E94B70A8093F90384E059
:102B20000E94B70A8093FA0387E061E00E94BD0A21
:102B30006AE070E080E090E00E94C9290E947C0C6D
:102B4000000008950F931F93082F17C02D9A64E675
:102B500070E080E090E00E94C9292D9864E670E062
:102B600080E090E00E94C9291F5F101778F36CE2A3
:102B700071E080E090E00E94C92910E0F6CF482F74
:102B8000392F25E00DC0F999FECF1FBA842F932F5E
:102B900092BD81BD60BD0FB6F894FA9AF99A0FBE46
:102BA000215059F0F999FECF842F932F92BD81BD0A
:102BB000F89A80B5681739F7089582E00E94A21547
:102BC0000895A0E0B0E0E7EEF5E10C94AE2F482EBA
:102BD000562ECC24DD24EE24FF2488249924C0E042
:102BE000D0E076E4372E04C0CC24DD245524539461
:102BF000442069F480919B03839DE00111246CE9DA
:102C0000E62E63E0F62E59E1852E912C1DC021E0C1
:102C1000421671F480919B03839DE00111246B9611
:102C200040EDE42E43E0F42E39E2832E912C0CC0CB
:102C300032E0431649F42BE9E22E23E0F22E91E034
:102C4000892E912CC8E1D1E03E016C0C7D1C1092C4
:102C5000320510923105E3011BC0552059F4F99952
:102C6000FECFD2BDC1BDF89A80B5F701E00FF11FCC
:102C7000808307C0F701E00FF11FCE0160810E9441
:102C8000BF150E0D1F1DF80180810E94300821968E
:102C90009E012619022F10E008151905F0F2CE0149
:102CA0005520D9F4F999FECFD2BDC1BDF89A20B50F
:102CB000F999FECF2196D2BDC1BD2197F89A80B572
:102CC00090E0B22EAA248A299B29209131053091C7
:102CD00032052817390759F487CF219660913205BC
:102CE0000E94BF15CE01609131050E94BF1580E2A0
:102CF00091E0C80ED91E91EEC91692E0D90608F4EB
:102D000077CF852DCDB7DEB7E1E10C94CA2F80E0F7
:102D100061E00E94E11581E061E00E94E115089503
:102D200080E060E00E94E115882331F081E060E0FE
:102D30000E94E115882331F40E9492080E944D08F8
:102D40000E948716089582E061E00E94E1150895CF
:102D500082E060E00E94E11580919B03843020F0C6
:102D600010929B030E94A31608951F93182F0E9490
:102D7000A81680919B03811731F0143020F4109332
:102D80009B030E94A3161F9108951092670485E685
:102D9000E2E0F4E0DF011D928A95E9F708951F93C0
:102DA000182F8F3711F08830E1F5E0916704EE239A
:102DB00009F455C0E150E0936704F0E0EE5FFB4F8B
:102DC000108285E396E06DE00E94AA2E10E00AC012
:102DD000E12FF0E0EE5FFB4F85E396E060810E941B
:102DE000AA2E1F5F80916704181790F385E396E081
:102DF00060E20E94AA2E85E396E06DE00E94AA2E72
:102E000010E00AC0E12FF0E0EE5FFB4F85E396E0B3
:102E100060810E94AA2E1F5F80916704181790F3AB
:102E20001CC08B3119F40E94C5161FC08D30E9F00B
:102E30008A30D9F080916704843688F485E396E07F
:102E4000612F0E94AA2E80916704E82FF0E0EE5FC8
:102E5000FB4F10838F5F8093670480E007C085E39A
:102E600096E067E00E945E2BF8CF81E01F91089505
:102E70001F93CF93DF93CFEDD3E010E03BC085E30A
:102E800096E062E271E00E94EF2C85E396E0612F0C
:102E90004AE050E00E946C2C85E396E06FE271E01E
:102EA0000E94EF2C699170E080E090E02091DE03B9
:102EB00030E040E050E00E943E2F20E137E240E069
:102EC00050E00E943E2FDC01CB014091D503509190
:102ED000D6036091D7037091D803480F591F6A1F1A
:102EE0007B1F85E396E02AE030E00E94332C1F5FD1
:102EF000183119F08881882311F6DF91CF911F9145
:102F00000895EF92FF920F931F93882339F485E37E
:102F100096E061E77AE00E947C2B3BC090E00E9443
:102F2000B20824E630E040E050E00E94702F122FFB
:102F3000032FF42EE52E622F732F842F952F2AE076
:102F400030E040E050E00E94702F85E396E0BA0147
:102F5000A9012AE030E00E94242C85E396E06EE28D
:102F60000E945E2B612F702F8F2D9E2D2AE030E066
:102F700040E050E00E94702FAB01BC0185E396E079
:102F80002AE030E00E94242C85E396E063E70E946B
:102F9000902B1F910F91FF90EF900895FF920F9348
:102FA0001F93CF93DF9385E396E067E67AE00E9474
:102FB0003D2B8091B503813041F485E396E06EE4CA
:102FC0007AE00E947C2BFF246DC0823029F485E3D7
:102FD00096E067E37AE0F5CF843029F485E396E064
:102FE00063E27AE0EECF853071F785E396E068E141
:102FF0007AE0E7CFCF2DD0E0C930D1051CF06F2D9E
:10300000685C02C06F2D6F5C85E396E00E945E2BCA
:1030100085E396E060E17AE00E943D2BBE016F5FA0
:103020007F4F85E396E04AE050E00E94C82C85E39C
:1030300096E065E07AE00E943D2B8E010B541C4F18
:10304000D8011196EC91E032F8F485E396E068EF50
:1030500079E00E943D2BF8018181803130F085E3D9
:1030600096E063E371E00E94EF2CCB54DC4F698162
:1030700070E06F7070706F5F7F4F85E396E04AE09D
:1030800050E00E94DB2C0DC0F0E0EF70F070EE0F0E
:10309000FF1FE75BFC4F6081718185E396E00E9432
:1030A000F22CF39480918A04F81608F4A3CF85E3F8
:1030B00096E06DED79E00E943D2B8091CD030E945A
:1030C000811785E396E062EC79E00E943D2B8091C8
:1030D000CE030E94811785E396E067EA79E00E94BB
:1030E0003D2B8091CF030E94811785E396E06CE829
:1030F00079E00E943D2B4091C5035091C603609139
:10310000C7037091C803411551056105710539F177
:1031100085E396E02AE030E00E94332C85E396E0D8
:1031200069E579E00E943D2B8091C9030E94E50882
:10313000AB01BC0185E396E02AE030E00E94332C2D
:1031400085E396E065E379E00E943D2B85E396E018
:103150006091CA034AE050E00E947E2C06C085E3DD
:1031600096E06CE279E00E947C2B85E396E06FE0CC
:1031700079E00E943D2B6091CB037091CC0385E3F5
:1031800096E04AE050E00E94582C85E396E062EF1A
:1031900078E00E943D2B6091C403603150F470E0F0
:1031A0006F5F7F4F85E396E04AE050E00E94DB2CA2
:1031B00006C085E396E069EE78E00E947C2B85E30B
:1031C00096E06CEC78E00E943D2B8091C30380FD7B
:1031D00003C065E371E002C069E371E085E396E056
:1031E0000E94F22C85E396E06FEA78E00E943D2B86
:1031F0008091C30382700E94930D85E396E060E99D
:1032000078E00E943D2B8091C30384700E94930D4F
:1032100085E396E061E778E00E943D2B8091C3034F
:1032200088700E94930DCDB7DEB7E5E00C94D62FE1
:103230001F93CF93DF9385E396E06BEB7BE00E94D7
:103240003D2B4091D5035091D6036091D7037091E7
:10325000D80385E396E02AE030E00E94332C85E332
:1032600096E065EA7BE00E943D2B4091D9035091A6
:10327000DA036091DB037091DC0385E396E020E1E3
:1032800030E00E94332C85E396E06FE87BE00E94FB
:103290003D2B85E396E06091DD034AE050E00E941B
:1032A0007E2C85E396E069E77BE00E943D2B85E379
:1032B00096E06091DE034AE050E00E947E2C85E3B8
:1032C00096E063E67BE00E943D2BCFEDD3E010E07B
:1032D00012C0112331F085E396E06DE371E00E94A6
:1032E000EF2C85E396E069914AE050E00E946C2C57
:1032F0001F5F183119F08881882359F785E396E01C
:103300000E94662B85E396E06DE47BE00E943D2BF6
:1033100085E396E06091F7034AE050E00E947E2C3E
:1033200085E396E068E37BE00E943D2BE091F803A3
:10333000F0E0E770F070EE0FFF1FE759FC4F60817F
:10334000718185E396E00E94F22C85E396E063E2CA
:103350007BE00E943D2B8091F80390E08871907093
:103360008830910589F0893091051CF4892B39F05A
:103370001BC08031910569F04897B1F40FC085E317
:1033800096E06AE17BE00EC085E396E06EE07BE0CC
:1033900009C085E396E068E07BE004C085E396E041
:1033A0006EEF7AE00E947C2B85E396E06AEE7AE08D
:1033B0000E943D2B4091D1035091D2036091D303E1
:1033C0007091D40385E396E02AE030E00E94332C2C
:1033D00085E396E061ED7AE00E943D2B8091A103A8
:1033E00080710E94930D85E396E068EB7AE00E947D
:1033F0003D2B8091A10380740E94930D85E396E09C
:103400006FE97AE00E943D2B8091A10380720E94B7
:10341000930D85E396E062E87AE00E943D2B80ED13
:1034200093E00E94F508AB01BC0185E396E02AE039
:1034300030E00E94242C85E396E06DE77AE00E945C
:103440003D2B80ED93E00E94F5089B01AC0160E408
:1034500072E48FE090E00E94702F85E396E0BA015D
:10346000A9012AE030E00E94242C85E396E06AE777
:103470007AE00E947C2BDF91CF911F910895EF920B
:10348000FF920F931F938C0195E3E92E96E0F92E9E
:10349000C701612F70E04AE050E00E94472CC7014D
:1034A0006EE20E945E2B84E0169507958A95E1F7FF
:1034B0000F701070C701B8014AE050E00E94472C1D
:1034C0001F910F91FF90EF9008950F931F93CF934B
:1034D000DF93209101042F3FA9F585E396E061EF8A
:1034E00075E00E943D2B80E793E00E943F1A85E340
:1034F00096E060ED75E00E943D2B80918B049091E9
:103500008C040E943F1A85E396E06DE975E00E9405
:103510007C2B85E396E06AE775E00E947C2B85E3CF
:1035200096E062E675E00E947C2B85E396E06DE311
:1035300075E00E947C2B85E396E00E94662B0E943A
:10354000CE1769C012160CF066C0332727FD3095E0
:1035500080918A0490E0821793070CF45CC085E3A5
:1035600096E068E275E00E943D2B609101047727A8
:1035700067FD709585E396E04AE050E00E94DB2C01
:1035800085E396E06DEF74E00E943D2B08E210E0C9
:103590003AC0C12FD0E0CC0FDD1FC759DB4F2881C7
:1035A00030E080910104992787FD909501972817B5
:1035B000390741F585E396E06FE371E00E94EF2C57
:1035C00085E396E0602F4AE050E00E946C2C85E392
:1035D00096E063E471E00E94EF2CE981F0E0EF7087
:1035E000F070EE0FFF1FE75BFC4F6081718185E398
:1035F00096E00E94EF2C85E396E067E471E00E947C
:10360000EF2C0F5F1F5F80918904181710F285E37C
:1036100096E00E94662BDF91CF911F910F91089544
:10362000ACE1B0E0E6E1FBE10C94B72F282F8091EC
:1036300001048F3F09F042C1822F90E0FC013A97CC
:10364000EF36F10508F033C1EC5CFF4F0C94E42F2A
:1036500085E396E069E471E0AEC085E396E069E455
:1036600071E00E94F22C1CC185E396E065E571E0F3
:103670000E94F22C85E78983DE011296E5EBF3E0E8
:103680008BE101900D928150E1F7CE0101966CE142
:103690000E94D70F0E947C0C83E080939A0368EC11
:1036A00070E080E090E00E94C92980919A03843004
:1036B00009F0FDC08FE70E94930A0E94A70A898340
:1036C000853509F0F4C085E396E06FED74E00E9463
:1036D0007C2B85E396E061EC74E00E947C2B85E313
:1036E00096E063EA74E0ACC085E396E06DE671E0D5
:1036F0000E94F22C89E68983CE01019661E00E9446
:10370000D70F0E947C0C83E080939A0368EC70E0F2
:1037100080E090E00E94C92980919A03843009F0EA
:10372000C6C08FE70E94930A0E94A70A89838E0170
:103730000E5F1F4FBDE1EB2EF12CEC0EFD1E0E9423
:10374000A70AD8018D938D01AE15BF05C1F7A5EB72
:10375000B3E0FE0132968BE101900D928150E1F7CA
:103760008981893409F0A3C085E396E065E874E0B7
:103770000E947C2B85E396E067E674E00E947C2B38
:1037800085E396E069E474E05BC085E396E067E872
:1037900071E00E94F22C8EEF8093010488C02052C9
:1037A0002750922F905380918A04891738F485E32B
:1037B00096E066E971E00E94F22C79C090930104D2
:1037C0006FC084E18093010485E396E062E174E0D8
:1037D00037C085E18093010485E396E06BED73E0EB
:1037E0002FC086E18093010485E396E064EA73E0EC
:1037F00027C087E18093010485E396E06AE573E0E2
:103800001FC088E18093010485E396E069E473E0DA
:1038100017C089E18093010485E396E065E373E0D6
:103820000FC08AE18093010485E396E060E273E0D3
:1038300007C08BE18093010485E396E068EF72E0B6
:103840000E947C2B34C085E396E06EED72E00E940E
:103850007C2B8091C30391E01DC085E396E068EC6A
:1038600072E00E947C2B8091C30392E013C085E339
:1038700096E063EB72E00E947C2B8091C30394E09E
:1038800009C085E396E068E972E00E947C2B809194
:10389000C30398E089278093C3038FEF80930104CB
:1038A0000E94651A04C085E396E00E94712E85E3AC
:1038B00096E00E94372E892BB1F762C1822F0E94B9
:1038C000CF16882309F45CC180916704882321F412
:1038D0008FEF809301044CC182E094E060E070E0DF
:1038E00040E050E00E94A2069B01AC0160910104FF
:1038F000862F992787FD9095A92FB92FFC01319725
:10390000EB31F10508F024C1ED55FF4F0C94E42F85
:10391000E62FFF27E7FDF09580918A0490E08E174F
:103920009F070CF415C1DA01C9010197A109B1097A
:103930008097A105B10548F0A8E2FA2E00E010E05A
:103940006F010894C108D10825C0EB54FC4F822FA9
:1039500081508083E5C0612F70E0660F771F675943
:103960007B4FFB01808190E08C159D0591F48F2D9C
:1039700090E0A0E0B0E082179307A407B50741F4F8
:10398000F601EB54FC4FDB0111968C91818301E031
:10399000F3941F5F809189041817E8F2BFC02F3F8E
:1039A00031054105510511F008F0D2C02093CD0337
:1039B000B7C02F3F31054105510511F008F0C8C0CF
:1039C0002093CE03ADC02F3F31054105510511F0C5
:1039D00008F0BEC02093CF03A3C080910204806290
:1039E000803719F583E094E060E070E040E050E05B
:1039F0000E94A2069B01AC01DC01CB010197A10949
:103A0000B1090897A105B10508F0B5C0CA01B9010F
:103A100024ED30E340E050E00E943E2F9B01AC01DA
:103A20002A5E3C4A4A46554E24C0863611F583E04C
:103A300094E060E070E040E050E00E94A2069B014C
:103A4000AC01DC01CB010197A109B1090797A105E0
:103A5000B10508F090C0CA01B90128EA31E640E09A
:103A600050E00E943E2F9B01AC01245E3C434E4639
:103A7000544E211531054105510561F0DA01C901A6
:103A800080509447AB48B24381509A45A246B24019
:103A900008F05EC02093C5033093C6034093C7036C
:103AA0005093C8033DC02F3F31054105510511F02A
:103AB00008F04EC02093C90333C0DA01C901019751
:103AC000A109B1098F3F9105A105B10508F040C0DA
:103AD0002093CA0325C0DA01C901845C9940A04043
:103AE000B0408D549D41A040B04030F43093CC03A1
:103AF0002093CB0301E001C000E021153105410511
:103B0000510511F48FEF07C02131310541055105F1
:103B100028F4822F81508093C40302C00023C1F097
:103B2000809168048823D1F48091D9039091DA03BD
:103B3000A091DB03B091DC030196A11DB11D809320
:103B4000D9039093DA03A093DB03B093DC0306C0A0
:103B500085E396E068EA71E00E94F22C0E94C516A7
:103B60008FEF8093010485E396E06AE00E94902B3A
:103B70000E94651A05C021E030E040E050E07ECFB1
:103B80006C96E8E00C94D32F85E396E06CE472E049
:103B90000E947C2B85E396E064E372E00E947C2B1C
:103BA00085E396E00E94372E892B31F085E396E07D
:103BB0000E94712E0E94101B0E94DE14823019F0A8
:103BC000833069F405C085E396E066E172E004C0E5
:103BD00085E396E06FEF71E00E947C2B08958FEFF4
:103BE00080930104109268040E94651A0CC085E35A
:103BF00096E00E94372E892B31F085E396E00E94F3
:103C0000712E0E94101B809101048E3F81F7089550
:103C100080910104992787FD9095A92FB92FFC0168
:103C20003196EB30F10508F074C0E254FF4F0C946C
:103C3000E42F85E396E064E678E00E947C2B80E741
:103C400093E00E943F1A85E396E06CE478E00E94DE
:103C50007C2B85E396E067E278E00E947C2B85E38D
:103C600096E06DEF77E00E947C2B85E396E06CEDAB
:103C700077E00E947C2B85E396E06FEA77E00E9474
:103C80007C2B85E396E069E877E00E947C2B85E356
:103C900096E065E677E00E947C2B85E396E06EE394
:103CA00077E00E947C2B85E396E00E94662B0E94C1
:103CB00018192FC085E396E061E277E028C085E31C
:103CC00096E06CEF76E023C085E396E067EE76E061
:103CD0001EC085E396E068EC76E019C085E396E0C7
:103CE00064E876E014C085E396E06FE676E00FC006
:103CF00085E396E06AE576E00E947C2B85E396E01A
:103D000064E176E004C085E396E06EEF75E00E9422
:103D10007C2B6AE070E080E090E00E94C92904C03A
:103D200085E396E00E94712E85E396E00E94372E8F
:103D3000892BB1F70895A2E2B0E0E1EAFEE10C942C
:103D4000AD2F8E010F5F1F4F80E1D8011D928A9524
:103D5000E9F785E396E066EC71E00E94F22C0E94A0
:103D60008A1520E034E74BE852E32F8F38A349A3AC
:103D70005AA380E09EECADEEB4E38B8F9C8FAD8FA9
:103D8000BE8F24EF31E040E050E02F8B388F498F19
:103D90005A8F30E5C32E33ECD32EE12CF12C412C7D
:103DA00024E7522E2BE8622E22E3722E88249924D7
:103DB000540133241E8A1D8A198A1A8A1B8A1C8A76
:103DC000FFC085E396E00E94712E8434B9F08534FB
:103DD00030F48332B9F18C3209F0CCC044C0833561
:103DE00009F0C8C02F8D38A149A15AA1C901DA0133
:103DF0002C013D01882499245401E2C085E396E01A
:103E000064E40E945E2B85E396E040E054E76BE8B3
:103E100072E32AE030E00E94922C85E396E06CE2A7
:103E20000E945E2B85E396E040E05EEC6DEE74E36D
:103E30002AE030E00E94922C85E396E06CE20E943A
:103E4000902BBEC019821A821B821C821D821E8288
:103E50001F82188619861A861B861C861D861E865A
:103E60001F86188A3AC0339434E0331609F0A8C08C
:103E700069817A818B819C8128EE33E040E050E0BB
:103E80000E943E2F6F8F78A389A39AA36D817E81B4
:103E90008F8198850E943E2F6B8F7C8F8D8F9E8F98
:103EA00089859A85AB85BC858F8B988FA98FBA8FB2
:103EB0006D857E858F8598890E943E2F6B017C01E0
:103EC00090E2C9169EE4D90690E0E90690E0F90672
:103ED00030F48CE162E30E94BD0A332471C0A0E398
:103EE000CA16A5E7DA06A0E0EA06A0E0FA0618F48A
:103EF0008CE162E2F0CFB0E4CB16BCE9DB06B0E0C7
:103F0000EB06B0E0FB0618F48CE166E2E4CFE0E5F6
:103F1000CE16E3ECDE06E0E0EE06E0E0FE0618F486
:103F20008CE162E1D8CFF0E6CF16FAEEDF06F0E0E2
:103F3000EF06F0E0FF0618F48CE165E1CCCF20E756
:103F4000C21621E1D20621E0E20620E0F20618F4D2
:103F50008CE161E0C0CF30EAC31636E8D30631E029
:103F6000E30630E0F30618F48CE163E0B4CF8CE1B3
:103F700065E0B1CF90ED292E280E49E0421500F101
:103F8000032D10E0000F111F000F111F81E090E0C2
:103F90008C0F9D1F080F191FD8016D917D918D9178
:103FA0009C912AE030E040E050E00E943E2F620DFC
:103FB000711D811D911DF80160837183828393833C
:103FC00085E396E00E94372E892B09F0FACE811402
:103FD0009104A104B10489F4C301B2010E94330B1E
:103FE00061E070E080E090E00E94C929FFEFFE8B65
:103FF0001D8A198A1A8A1B8A1C8A2F89388D498D35
:104000005A8D82169306A406B506E0F40E94DE0AD5
:1040100029893A894B895C89280F311D411D511D21
:10402000298B3A8B4B8B5C8B3D89381708F48D8B31
:104030004E89841708F48E8B0894811C911CA11C56
:10404000B11C56C0C301B20128EE33E040E050E09D
:104050000E94702F85E396E0BA01A9012AE030E0C2
:104060000E94242C85E396E06CE20E945E2B85E39F
:1040700096E06D894AE050E00E946C2C85E396E062
:104080006CE20E945E2B69897A898B899C89A501E3
:1040900094010E94702F85E396E0BA01A9012AE0FD
:1040A00030E00E94242C85E396E06CE20E945E2BB7
:1040B00085E396E06E894AE050E00E946C2C85E32F
:1040C00096E06CE20E94902B4C0C5D1C6E1C7F1CD9
:1040D0008B8D9C8DAD8DBE8D84159505A605B70580
:1040E00020F44F8C58A069A07AA088249924540108
:1040F0002F8D38A149A15AA1285E3340404050403D
:1041000009F05ECFA296E2E10C94C92FAAE5B0E0D7
:10411000ECE8F0E20C94B92F8B017A018B3009F4B2
:1041200026C18C3040F5853009F484C0863080F497
:10413000823009F459C0833020F4813009F052C232
:1041400042C0833009F461C0843009F04BC265C0BD
:10415000883009F49DC0893038F4863009F486C06F
:10416000873009F03FC28CC0893009F499C08A3089
:1041700009F038C2C9C0893609F484C18A3680F48E
:10418000863609F42FC1873620F4853609F02AC215
:1041900010C1873609F43FC1883609F023C243C1F4
:1041A0008C3609F4C6C18D3638F48A3609F475C1E7
:1041B0008B3609F017C2B1C18D3609F4EEC1873CC8
:1041C00009F010C202C281E069E270E00E948F1122
:1041D00000ED13E0F80181918F010E947811F3E066
:1041E000093F1F07B9F706C282E06BE170E00E9449
:1041F0008F1105EB13E0F80181918F010E94781176
:10420000F3E0003D1F07B9F7F5C183E061E070E01E
:104210000E948F110E94DE14EBC184E061E070E027
:104220000E948F1181E00E9478110E9471110E94FA
:104230009B1EE2C16091890470E0660F771F85E0E4
:104240000E948F1100E010E008C0F801E759FB4F11
:1042500080810E9478110F5F1F4F8091890490E048
:10426000880F991F0817190780F3C4C186E062E020
:1042700070E00E948F1180E793E00E948611BAC11E
:1042800087E061E070E00E948F1180918A04B0C1E4
:1042900088E061E070E00E948F1180919B03A8C1CB
:1042A00086E68983CE01019661E00E94D70F0E94C5
:1042B0007C0C83E080939A0368EC70E080E090E0EF
:1042C0000E94C92980919A038430E1F48FE70E940B
:1042D000930A0E94A70A8983863471F489E060E218
:1042E00070E00E948F1110E00E94A70A0E947811CE
:1042F0001F5F1032C9F77EC189E061E070E00E9463
:104300008F11C9C089E06FC18AE069E170E00E9445
:104310008F1181E080939C0380919F05882351F049
:104320008091A1039091A203A091A303B091A40353
:10433000806809C08091A1039091A203A091A3037A
:10434000B091A4038F778093A1039093A203A093CD
:10435000A303B093A4030CE913E0F80181918F014A
:104360000E947811F3E0053B1F07B9F743C18BE0CA
:1043700061E270E00E948F118091BE048F3F39F09E
:104380008091BE048F5F8093BE04815002C08091F3
:10439000BE040E94781110E0F894812F0E94AE11A3
:1043A0000E94190A0E94861178941F5F1031A1F7AC
:1043B00021C185E661E070E00E948F11093211058C
:1043C00009F015C120E030E0F901E053FC4FD701BE
:1043D000A20FB31F8C9180832F5F3F4F293231058D
:1043E00099F759C086E661E070E00E948F110B31A9
:1043F000110509F0FCC020E030E0F901EB54FC4F5E
:10440000D701A20FB31F8C9180832F5F3F4F2B31B9
:10441000310599F740C087E661E070E00E948F1196
:104420000E94871638C088E661E070E00E948F1114
:1044300085E78A83DE011396E5EBF3E08BE10190DB
:104440000D928150E1F7CE0102966CE10E94D70FE8
:104450000E947C0C83E080939A0360E273E080E02A
:1044600090E00E94C92980919A03843009F0BFC06E
:104470008FE70E94930A0E94A70A8A83853509F074
:10448000B6C009C089E661E070E00E948F110E9409
:104490004D080E94920881E0ABC08AE661E070E0BE
:1044A0000E948F1189E68E8FCE014E9661E00E94A8
:1044B000D70F0E947C0C83E080939A0360E273E044
:1044C00080E090E00E94C92980919A03843009F02D
:1044D0008EC08FE70E94930A0E94A70A8E8F8E01DA
:1044E000015E1F4F4AE3E42EF12CEC0EFD1E0E94EC
:1044F000A70AF80181938F01EE15FF05C1F7A5EB1F
:10450000B3E0FE017F968BE101900D928150E1F7BF
:104510008E8D893409F06BC0BECF8BE661E070E010
:104520000E948F11F70180810E94B5160E9490169B
:10453000B2CF8CE661E070E00E948F11003211056D
:1045400071F487E68AAFDE01DB96F70180E2019025
:104550000D928150E1F7CE01CA9661E205C087E471
:104560008AAFCE01CA9661E00E94D70F0E947C0CF0
:1045700083E080939A036CE474E080E090E00E9412
:10458000C92980919A03843091F58FE70E94930A9C
:104590000E94A70A873459F57ECF8DE661E070E06E
:1045A0000E948F110931110511F520E030E0F90169
:1045B000E456FC4FD701A20FB31F8C9180832F5F6D
:1045C0003F4F2931310599F766CF87EC61E070E004
:1045D0000E948F1181E00E9478110E947111109247
:1045E000FF030AC08AEC61E070E00E948F1180E056
:1045F0000E9478110E947111C65ADF4FE6E00C94B8
:10460000D52FA0E0B0E0E7E0F3E20C94B52F84E012
:10461000A82E06E0B02E15E0C12E03E315E0B4E6A7
:10462000DB2EA2E0EA2EF3E0FF2EA1C085E396E0A8
:104630000E94712E982F80939E0580919D05833056
:1046400021F1843028F4813099F08230B8F409C027
:10465000853009F448C0853020F1863009F087C0E4
:104660005FC0953B09F083C081E080939D057FC0CA
:10467000923609F07AC0E0929D0579C090939C052E
:1046800090939B05F0929D0572C0909399051092AE
:104690009A0580919B05892780939B05A0929D0593
:1046A00066C0D92FC0E02091990530919A052C2B36
:1046B0003D2B30939A052093990580919B0589277E
:1046C00080939B05C0929D052536310508F44FC0A7
:1046D0008CEC61E070E00E948F1181E00E94781103
:1046E0000E94711142C02091970530919805F901FF
:1046F000ED5CFA4F908380919B05892780939B0501
:104700002F5F3F4F3093980520939705809199052F
:1047100090919A052817390750F1B0929D0527C04E
:1047200080919B05891759F46091970570919805C0
:1047300080919C0543E355E00E9486200DC08BECE0
:1047400062E070E00E948F1180919C050E947811B8
:10475000809100040E947811F8018D2D11928A95A4
:10476000E9F7109298051092970510929D0585E340
:1047700096E00E94372E892B09F058CFCDB7DEB7CF
:10478000EAE00C94D12F81E08093FF0308C085E319
:1047900096E00E94372E892B11F00E940123809110
:1047A000FF038823A1F70895A0E0B0E0EAEDF3E26B
:1047B0000C94B82F0E94A3296115710581059105FC
:1047C000C9F30E9499061092D9031092DA0310924D
:1047D000DB031092DC03DD24E090D903F090DA03D0
:1047E0000091DB031091DC03102F0F2DFE2CEE2423
:1047F0000E9494062FEF30E040E050E00E94922F9C
:10480000E60EF71E081F191FE092D903F092DA0393
:104810000093DB031093DC03D39444E0D416E1F659
:10482000CFEDD3E000E010E090E1E92E97E2F92E21
:104830004EC00F5F19F40E944D084DC00E949406AF
:1048400022E330E040E050E00E94922F6F5FEFEDF6
:10485000F3E090E004C08191861759F39F5F9117B0
:10486000D0F38091DE0390E08E9D90018F9D300DFE
:104870009E9D300D1124862F90E0AC01249FC00135
:10488000259F900D349F900D1124AA2797FDA09588
:10489000BA2F2091D5033091D6034091D703509180
:1048A000D803820F931FA41FB51F20919D03309141
:1048B0009E0340919F035091A003281739074A0790
:1048C0005B0708F4B6CF69931F5F183121F0888128
:1048D000882309F0AECFCDB7DEB7E7E00C94D42F34
:1048E0001F93109101041F3F09F0F1C0893409F4AE
:1048F00067C08A3428F5883309F479C0893368F4AD
:10490000803309F486C0813308F06FC08B3109F41D
:104910004DC0813209F0D5C03DC0813409F49AC040
:10492000823438F4893309F472C0803409F0C9C084
:1049300031C0823409F4A1C0863409F0C2C052C02B
:10494000823609F49AC0833690F4883579F1893536
:1049500038F4823509F43FC0833509F0B2C01FC076
:104960008A3509F4A9C0813609F0ABC073C082371B
:1049700091F1833730F48636A9F1893609F0A1C068
:104980001FC0883799F08A3709F496C0833709F039
:1049900098C005C085E396E069E471E019C00E9403
:1049A000871685E396E063ED71E006C00E949016DD
:1049B00085E396E06DEE71E00E94F22C8EEF7FC0F1
:1049C0000E944D080E94920885E396E06CE072E038
:1049D0000E94F22C76C00E94D42385E396E065E223
:1049E00072E0F6CF0E9438176CC0805368C085E330
:1049F00096E06CEE71E00E947C2B9091F803892F79
:104A0000885F8871977E892B8093F80320C089E0A6
:104A100056C085E396E069ED71E00E947C2B8091A1
:104A2000A1039091A203A091A303B091A40320E15C
:104A300030E040E050E082279327A427B5278093F9
:104A4000A1039093A203A093A303B093A403109394
:104A5000010437C085E396E063EC71E00E947C2B93
:104A60008091A1039091A203A091A303B091A4030C
:104A700020E430E040E050E012C085E396E062EBD5
:104A800071E00E947C2B8091A1039091A203A091E0
:104A9000A303B091A40320E230E040E050E082277D
:104AA0009327A427B5278093A1039093A203A093F3
:104AB000A303B093A40302C00E94C41D8FEF809390
:104AC0000104809101048E3F09F4DDC0D4C00E942E
:104AD000CF16882309F4D7C080916704882321F476
:104AE0008FEF80930104C7C082E094E060E070E043
:104AF00040E050E00E94A2069B01AC0180910104BD
:104B0000992787FD9095A92FB92FFC013197E9309E
:104B1000F10508F08CC0E753FF4F0C94E42FDA0145
:104B2000C90181509447AB48B2438F5F9945A24673
:104B3000B24008F07CC02093D5033093D603409355
:104B4000D7035093D8039AC02093D9033093DA0344
:104B50004093DB035093DC0381E0809368048EC0B4
:104B6000283031054105510508F061C02093DD036F
:104B700085C0DA01C9010197A109B1090A97A10508
:104B8000B10508F054C02093DE0378C082E094E0C1
:104B90006DE371E00E94BE0710E00EC0183130F4E2
:104BA000E12FF0E0E053FC4F87871F5F80E090E04B
:104BB0006DE371E00E94BE07009759F00E94A007C4
:104BC000009761F706C0E12FF0E0E053FC4F178635
:104BD0001F5F1831C0F352C0253031054105510522
:104BE00030F52093F7034AC0DA01C9010197A10902
:104BF000B1090697A105B105D0F48091F803887F2B
:104C0000822B8093F8033AC0DA01C9010197A10908
:104C1000B1098050924CA140B04048F42093D10398
:104C20003093D2034093D3035093D40327C085E33A
:104C300096E068EA71E00E94F22C13C08091D903DB
:104C40009091DA03A091DB03B091DC030196A11DE2
:104C5000B11D8093D9039093DA03A093DB03B09343
:104C6000DC030E94C5168FEF8093010485E396E074
:104C70006AE00E94902B0E94081E05C08091680483
:104C80008823E1F2EECF1F9108958FEF8093010406
:104C9000109268040E94081E0CC085E396E00E94F2
:104CA000372E892B31F085E396E00E94712E0E9409
:104CB0007024809101048E3F81F76AE070E080E00B
:104CC00090E00E94C92904C085E396E00E94712EFD
:104CD00085E396E00E94372E892BB1F70895AAE26A
:104CE000B0E0E5E7F6E20C94B22F0E9495297B0133
:104CF0008C0181E00E949D0B04C085E396E00E9438
:104D0000712E85E396E00E94372E892BB1F72D98FE
:104D1000DD24D39452E6752E42E0842E912C8C0E25
:104D20009D1E5E010894A11CB11C33E0C32E0E949D
:104D3000952920E030E06E197F09800B910B693CCA
:104D400071058105910510F021E030E08D2D90E096
:104D500028233923232B99F10E9495297B018C016B
:104D60002C9A80ED97E00E94E2117982D401E0ED67
:104D7000F3E089E201900D928150E1F7C5016AE20A
:104D80000E94D70F2C9880E090E00E94E211C09220
:104D90009A030E947C0C62E370E080E090E00E9445
:104DA000C92980919A03843051F4C0929A038FE705
:104DB0000E94930A0E94A70A823409F4DD248BE042
:104DC0000E94C72A892B49F5DD24D39426C02D9A49
:104DD0002C9A85E396E00E94712E8D30910569F042
:104DE0008E3091051CF40A97B1F407C08332910507
:104DF00069F08234910579F40CC085E396E064EAA9
:104E000071E00E947C2B0E94452605C00E949B1EDB
:104E100002C00E94C3232D982C9885E396E00E943F
:104E2000372E892B09F483CFD2CF8F929F92AF92E6
:104E3000BF92CF92DF92EF92FF920F931F938BE07E
:104E40000E94C72A892B09F083C068EC70E080E0DB
:104E500090E00E94C92980E090E00E94E2110E9447
:104E600095295B016C0160ECE62E62E1F62E012DC6
:104E7000112DEA0CFB1C0C1D1D1D06C08BE00E94B1
:104E8000C72A892B09F062C00E9495296E157F05FB
:104E90008007910798F38BE00E94C72A892B09F0BD
:104EA00055C080ED97E00E94E2110E9495297B0198
:104EB0008C0199249394882488E496E2A0E0B0E0E1
:104EC000A80EB91ECA1EDB1E29C0AE14BF04C00640
:104ED000D10638F480ED97E00E94E2118824839493
:104EE0001DC00E9495296E197F09800B910B693CAA
:104EF00071058105910590F00E9495297B018C0137
:104F000080E0992009F481E0982E882319F480E04C
:104F100090E002C080ED97E00E94E2118BE00E94D9
:104F2000C72A892B91F280E090E00E94E21188204C
:104F300049F080919B038F5F83700E94B5160E9499
:104F4000901606C00E94D4230E9487160E946F26E6
:104F50001F910F91FF90EF90DF90CF90BF90AF9097
:104F60009F908F90089580E06DEF77E042E050E0F1
:104F70000E94D0280895EF92FF920F931F9380E034
:104F80000E9419080E94CD118DE061E00E94282A3C
:104F90008CE061E00E94282A8BE060E00E94282AD1
:104FA00083E060E00E94282A83E061E00E94942A66
:104FB0008EE061E00E94282A8EE060E00E94942A40
:104FC0000E94B61485E396E040E052EC61E070E0A8
:104FD0000E94B02D0E94A8160E9490160E94720D89
:104FE0008FEF8093BE040E94B32778940E94952986
:104FF0007B018C018091BE048F3F09F0C7C00E94E5
:1050000095296E197F09800B910B605D7740804078
:10501000904008F0BBC0EECF85E396E00E94712E71
:1050200085E396E00E94372E892BB1F785E396E061
:1050300062E472E00E94EF2C80E793E00E943F1A46
:1050400085E396E069E572E00E94EF2C85E396E047
:1050500062E070E04AE050E00E94DB2C62E370E026
:1050600080E090E00E94C92985E396E00E94372EF7
:1050700004970CF185E396E00E94712E823491052D
:10508000D1F485E396E00E94712E8E34910599F457
:1050900085E396E00E94712E8434910561F485E3E6
:1050A00096E00E94712E819731F480E090E00E949A
:1050B000E2110E946F264091D1035091D20360917A
:1050C000D3037091D403DB01CA010197A109B1098F
:1050D0000497A105B10568F44093BF04433029F05B
:1050E00040E052EC61E070E004C040EA56E861E064
:1050F00070E085E396E00E94B02D0E9415272D9860
:1051000080E090E00E94E2110E94720D80E00E9417
:105110009D0B8091A4040E94C80A0E947C0C1092EE
:105120002705109228051092290510E015C062E3AA
:1051300070E080E090E00E94C92980ED97E00E9435
:10514000E21162E370E080E090E00E94C92980E013
:1051500090E00E94E2111F5F80919B03811738F756
:105160008091F80390E084FF09C020E0887190707E
:10517000489709F421E0822F0E94BF148FE00E941B
:1051800019081F910F91FF90EF90089580ED97E01F
:105190000E94E2118BE061E00E94942A2D9A40CF98
:1051A000823000F5E82FF0E0EE0FFF1FE056FA4FD7
:1051B00071836083882319F08130A1F408C0809145
:1051C00069008C7F842B80936900E89A0895809110
:1051D0006900440F551F440F551F837F842B809314
:1051E0006900E99A08951F920F920FB60F92112449
:1051F0002F933F934F935F936F937F938F939F93DF
:10520000AF93BF93EF93FF938091A0059091A10579
:10521000892B29F0E091A005F091A1050995FF9156
:10522000EF91BF91AF919F918F917F916F915F911E
:105230004F913F912F910F900FBE0F901F90189597
:105240001F920F920FB60F9211242F933F934F93FB
:105250005F936F937F938F939F93AF93BF93EF93DE
:10526000FF938091A2059091A305892B29F0E091ED
:10527000A205F091A3050995FF91EF91BF91AF9120
:105280009F918F917F916F915F914F913F912F915E
:105290000F900FBE0F901F9018951F920F920FB690
:1052A0000F9211242F933F938F939F93AF93BF93AC
:1052B0008091A8059091A905A091AA05B091AB0590
:1052C0003091AC050196A11DB11D232F2D5F2D3707
:1052D00020F02D570196A11DB11D2093AC058093A0
:1052E000A8059093A905A093AA05B093AB0580915A
:1052F000A4059091A505A091A605B091A7050196DA
:10530000A11DB11D8093A4059093A505A093A605AA
:10531000B093A705BF91AF919F918F913F912F912E
:105320000F900FBE0F901F9018958FB7F894209193
:10533000A8053091A9054091AA055091AB058FBFF2
:10534000B901CA0108959FB7F8942091A40530913E
:10535000A5054091A6055091A70586B5A89B06C056
:105360008F3F21F02F5F3F4F4F4F5F4F9FBF542F15
:10537000432F322F2227280F311D411D511D82E05E
:10538000220F331F441F551F8A95D1F7B901CA0157
:105390000895EF92FF920F931F93CF93DF937B01BA
:1053A0008C010E94A329EB010EC00E94A3296C1B53
:1053B0007D0B685E7340C8F30894E108F1080109A9
:1053C0001109C851DC4FE114F1040105110569F719
:1053D000CDB7DEB7E6E00C94D52F789484B5826023
:1053E00084BD84B5816084BD85B5826085BD85B589
:1053F000816085BDEEE6F0E0808181608083E1E838
:10540000F0E010828081826080838081816080836F
:10541000E0E8F0E0808181608083E1EBF0E0808172
:1054200084608083E0EBF0E0808181608083EAE744
:10543000F0E08081846080838081826080838081CD
:10544000816080838081806880831092C10008958C
:10545000CF93DF93482F50E0CA018D5F934FFC013B
:1054600034914151544FFA018491882369F190E0BD
:10547000880F991FFC01EF52F44FA591B491FC01E4
:10548000E552F44FC591D491662351F42FB7F894A7
:105490008C91932F909589238C93888189230BC0BD
:1054A000623061F42FB7F8948C91932F90958923F3
:1054B0008C938881832B88832FBF06C09FB7F89475
:1054C0008C91832B8C939FBFDF91CF910895833074
:1054D00071F0843028F48130A1F0823021F514C0BD
:1054E0008630B1F08730D1F08430E9F404C0809187
:1054F00080008F7703C0809180008F7D8093800033
:10550000089584B58F7702C084B58F7D84BD0895DA
:105510008091B0008F778093B00008958091B000A3
:105520008F7D8093B0000895FF920F931F93F62E06
:10553000482F50E0CA01895E934FFC012491CA01B3
:105540008D5F934FFC0114914151544FFA01049126
:105550000023C9F0222319F0822F0E94672AE02F2E
:10556000F0E0EE0FFF1FE552F44FA591B4919FB705
:10557000F894FF2021F48C911095812302C08C9126
:10558000812B8C939FBF1F910F91FF9008950F93D4
:105590001F93482F50E0CA01895E934FFC0124916C
:1055A000CA018D5F934FFC0104914151544FFA01A0
:1055B0001491112319F420E030E015C0222319F0D2
:1055C000822F0E94672A812F90E0880F991F8B51AC
:1055D000944FFC01A591B4918C9120E030E08023A0
:1055E00011F021E030E0C9011F910F910895982F2B
:1055F0008E3008F09E509770809148038295880FF6
:10560000880F807C892B80937C0080917A00806455
:1056100080937A0080917A0086FDFCCF20917800FB
:1056200040917900942F80E030E0282B392BC9017C
:105630000895A0E0B0E0EFE1FBE20C94B72F7C010D
:105640006B018A01C0E0D0E00FC0D6016D916D0101
:10565000D701ED91FC910190F081E02DC7010995F2
:10566000C80FD91F015010400115110571F7CE0167
:10567000CDB7DEB7E8E00C94D32FEF92FF920F93F3
:105680001F93CF93DF937C018B01C0E0D0E0F80142
:105690000F5F1F4F6491662359F0D701ED91FC9184
:1056A0000190F081E02DC7010995C80FD91FEFCFF8
:1056B000CE01CDB7DEB7E6E00C94D52FDC01ED913D
:1056C000FC910190F081E02D09950895EF92FF92F1
:1056D0000F931F938C016DE00E945E2B7C01C8012B
:1056E0006AE00E945E2B9C012E0D3F1DC9011F9197
:1056F0000F91FF90EF900895EF92FF920F931F93F9
:105700007C010E943D2B8C01C7010E94662B9C01ED
:10571000200F311FC9011F910F91FF90EF90089545
:10572000EF92FF920F931F937C010E945E2B8C01DE
:10573000C7010E94662B9C01200F311FC9011F91D8
:105740000F91FF90EF900895CF93DF93EC016115D7
:10575000710519F420E030E00FC0DB010D9000204E
:10576000E9F71197A61BB70BE881F9810280F38155
:10577000E02DAD0109959C01C901DF91CF910895FC
:105780004F925F927F928F929F92AF92BF92CF92F1
:10579000DF92EF92FF920F931F93DF93CF93CDB7DA
:1057A000DEB7A1970FB6F894DEBF0FBECDBF2C01B8
:1057B000742ECB01223008F42AE019A231E2C32E64
:1057C000D12CCC0EDD1E822E9924AA24BB24672D59
:1057D000752FA50194010E94702F79018A01C801DB
:1057E000B701A50194010E943E2F472D461B089446
:1057F000C108D1084A3010F4405D01C0495CF6018F
:105800004083E114F1040105110521F07E2C5F2D88
:10581000C801DDCFC201B6010E94A42BA1960FB62C
:10582000F894DEBF0FBECDBFCF91DF911F910F91D6
:10583000FF90EF90DF90CF90BF90AF909F908F90B0
:105840007F905F904F900895DC012115310541F460
:10585000ED91FC910190F081E02D642F0995089560
:105860000E94C02B0895EF92FF920F931F937C012B
:105870000E94242C8C01C7010E94662B9C01200FE2
:10588000311FC9011F910F91FF90EF900895EF9282
:10589000FF920F931F939A017B0100E010E0B80183
:1058A000A7010E94242C1F910F91FF90EF90089563
:1058B000EF92FF920F931F937C010E94472C8C0163
:1058C000C7010E94662B9C01200F311FC9011F9147
:1058D0000F91FF90EF900895EF92FF920F931F9317
:1058E0009A01E62EFF2400E010E0B801A7010E9413
:1058F000242C1F910F91FF90EF900895EF92FF924B
:105900000F931F937C010E946C2C8C01C7010E9495
:10591000662B9C01200F311FC9011F910F91FF9031
:10592000EF900895A0E0B0E0E8E9FCE20C94B72F16
:10593000EC016A017B012115310541F4E881F9810F
:105940000190F081E02D642F09951BC02A303105AC
:10595000B1F477FF13C06DE20E945E2B8C014427E7
:105960005527BA014C195D096E097F09CE012AE05D
:105970000E94C02B9C01200F311F04C02AE00E940E
:10598000C02B9C01C901CDB7DEB7E8E00C94D32F42
:10599000EF92FF920F931F937B019A010027F7FC70
:1059A0000095102FB801A7010E94922C1F910F9112
:1059B000FF90EF900895EF92FF920F931F937C0159
:1059C0000E94C82C8C01C7010E94662B9C01200FED
:1059D000311FC9011F910F91FF90EF9008950E9410
:1059E000A42B0895EF92FF920F931F937C010E94C6
:1059F000EF2C8C01C7010E94662B9C01200F311FE8
:105A0000C9011F910F91FF90EF90089508951F9283
:105A10000F920FB60F9211242F933F934F938F93B2
:105A20009F93EF93FF938091C00082FD1DC0409132
:105A3000C6002091ED053091EE052F5F3F4F2F738B
:105A400030708091EF059091F0052817390771F0BB
:105A5000E091ED05F091EE05E355FA4F4083309368
:105A6000EE052093ED0502C08091C600FF91EF91F5
:105A70009F918F914F913F912F910F900FBE0F905B
:105A80001F9018951F920F920FB60F9211242F930B
:105A90003F938F939F93EF93FF9320913106309123
:105AA000320680913306909134062817390731F475
:105AB0008091C1008F7D8093C10014C0E0913306B6
:105AC000F0913406EF50FA4F208180913306909187
:105AD000340601968F73907090933406809333064A
:105AE0002093C600FF91EF919F918F913F912F914D
:105AF0000F900FBE0F901F901895A0E0B0E0E3E864
:105B0000FDE20C94B32FFC011382128288EE93E025
:105B1000A0E0B0E084839583A683B7838BE893E00D
:105B2000918380837587648757874687318B208B65
:105B3000138B028BF58AE48AD78AC68AB18EA08E2F
:105B4000938E828E8F85848F8889858F8989868FB1
:105B50008A89878F8B8980A32096ECE00C94CF2FC5
:105B6000AF92BF92DF92EF92FF920F931F93CF936A
:105B7000DF93EC017A018B01DD24403081EE580780
:105B800080E0680780E0780711F0DD24D39491E08D
:105B9000A92EB12CEC89FD89DD2069F0C50108A092
:105BA00002C0880F991F0A94E2F7808360E079E0D1
:105BB0008DE390E005C0108260E874E88EE190E02B
:105BC000A80197010E94702F215030404040504062
:105BD000569547953795279580E12030380720F076
:105BE000DD2011F0DD24D6CFE889F9893083EA89F8
:105BF000FB89208319A2EE89FF89408121E030E0F2
:105C0000C9010C8C02C0880F991F0A94E2F7482B37
:105C10004083EE89FF894081C9010D8C02C0880F45
:105C2000991F0A94E2F7482B4083EE89FF8940814F
:105C3000C9010E8C02C0880F991F0A94E2F7482B05
:105C40004083EE89FF8980810F8C02C0220F331FB1
:105C50000A94E2F7209528232083DF91CF911F91AA
:105C60000F91FF90EF90DF90BF90AF900895DC010F
:105C70001C96ED91FC911D97E05CFF4F21913191B5
:105C800080819181281B390B2F733070C9010895D1
:105C900085E396E00E94372E892B11F00E94062D95
:105CA0000895DC011C96ED91FC911D97E05CFF4F7F
:105CB00020813181E054F040DF01AE5BBF4F8D9118
:105CC0009C9111972817390719F42FEF3FEF07C060
:105CD0008D919C91E80FF91F8081282F30E0C90138
:105CE0000895DC011C96ED91FC911D97E05CFF4F3F
:105CF00020813181E054F040DF01AE5BBF4F8D91D8
:105D00009C9111972817390719F42FEF3FEF10C016
:105D10008D919C911197E80FF91F20818D919C9195
:105D2000119701968F73907011969C938E9330E02B
:105D3000C9010895DC0191968C919197882339F0DF
:105D40005496ED91FC915597808186FFF9CF9196FD
:105D50001C920895CF93DF93EC01EE85FF85E05C04
:105D6000FF4F20813181E054F0402F5F3F4F2F7370
:105D70003070DF01AE5BBF4F8D919C91119728175A
:105D80003907D1F3E05CFF4F80819181E054F0400E
:105D9000E80FF91F6083EE85FF85E05CFF4F3183DC
:105DA0002083EE89FF89208181E090E00F8C02C082
:105DB000880F991F0A94E2F7282B208381E089A39A
:105DC000EC89FD8980818064808381E090E0DF91AF
:105DD000CF9108958F929F92AF92BF92CF92DF9210
:105DE000EF92FF920F931F9300D000D00F92EDB768
:105DF000FEB7319684E0ADB7BEB711968C9383E0C1
:105E0000818387E0828385E0838381E0848385E3E7
:105E100096E06DEA75E041EF55E025EC30E004ECEA
:105E200010E0B0ECEB2EF12CA1ECCA2ED12CF2EC50
:105E3000AF2EB12CE6EC8E2E912C0E947D2D0F9072
:105E40000F900F900F900F901F910F91FF90EF9078
:105E5000DF90CF90BF90AF909F908F900895CF9399
:105E6000DF930E94ED290E94BB27C8E4DEE20E9476
:105E7000EC112097E1F30E94482EF9CF629FD001E8
:105E8000739FF001829FE00DF11D649FE00DF11DF5
:105E9000929FF00D839FF00D749FF00D659FF00DA4
:105EA0009927729FB00DE11DF91F639FB00DE11D91
:105EB000F91FBD01CF011124089597FB092E072674
:105EC0000AD077FD04D086D006D000201AF4709551
:105ED00061957F4F0895F6F7909581959F4F0895AE
:105EE000A1E21A2EAA1BBB1BFD010DC0AA1FBB1FDE
:105EF000EE1FFF1FA217B307E407F50720F0A21B50
:105F0000B30BE40BF50B661F771F881F991F1A94BC
:105F100069F760957095809590959B01AC01BD01E6
:105F2000CF01089597FB092E05260ED057FD04D00A
:105F3000D7DF0AD0001C38F4509540953095219554
:105F40003F4F4F4F5F4F0895F6F7909580957095AE
:105F500061957F4F8F4F9F4F08952F923F924F92A1
:105F60005F926F927F928F929F92AF92BF92CF92E9
:105F7000DF92EF92FF920F931F93CF93DF93CDB7F2
:105F8000DEB7CA1BDB0B0FB6F894DEBF0FBECDBF6A
:105F900009942A88398848885F846E847D848C843B
:105FA0009B84AA84B984C884DF80EE80FD800C8144
:105FB0001B81AA81B981CE0FD11D0FB6F894DEBF27
:105FC0000FBECDBFED010895EE0FFF1F0590F491B8
:105FD000E02D0994AA1BBB1B51E107C0AA1FBB1FE0
:105FE000A617B70710F0A61BB70B881F991F5A9565
:105FF000A9F780959095BC01CD010895911106C037
:10600000803219F089508550D0F708959927882754
:066010000895F894FFCF93
:106016004E6F005965730054582074696D656F752D
:106026007421006D6F64756C65206C6F636B6564BD
:106036003F00486F70206368616E6E656C200020BB
:1060460040200053004E2F4100386368002C002C7E
:10605600205B005D20280029004E4F5420454E410C
:10606600424C45440053656E64696E6720736574DF
:1060760074696E677320746F2052580A00526573F4
:10608600657474696E672073657474696E677320CE
:106096006F6E2052580A0041626F72746564206503
:1060A600646974730A00696E76616C69642073654D
:1060B6006C656374696F6E000D0A496E76616C6972
:1060C6006420696E707574202D2064697363617233
:1060D6006465642107007363616E6E6572206D6F7F
:1060E60064650053657474696E67732073617665C1
:1060F6006420746F20454550524F4D0A0052657614
:1061060065727465642073657474696E677320665E
:10611600726F6D20454550524F4D0A004C6F6164B9
:10612600656420666163746F727920646566617563
:106136006C74730A004B657920616E642063686134
:106146006E6E656C732072616E646F6D697A6564DC
:106156000A004F70656E4C52536E67205458207378
:1061660074617274696E672000206F6E2048572034
:106176000050504D0052535349005344410053437D
:106186004C00525844005458440041494E004C4279
:106196004545500053504B54524D00534255530001
:1061A60053554D44004C4C494E440000342B3400AA
:1061B6003800382B340031320031322B340031367E
:1061C6000001000000C01200001A400AA1204EA5DE
:1061D600001B1E27522C23308025000005400AA1F3
:1061E600204EA50020244EA52C2330004B0000068F
:1061F600400AD0009D49007B289D492C233000E1B0
:10620600000005400A4501D7DC03B81E0EBF002377
:106216002E48E801008A400A6001555502AD1E204D
:10622600000023C88025000005400AA1204EA500D5
:1062360020244EA52C23300002000200020002009A
:106246000200020002000200020002000200020038
:1062560002000200020002FF01610265026A026E8C
:1062660002720276027A027E0284028B0290029504
:10627600029B029B029B029B0235019C02A002A28A
:1062860002A602A902AE02350100070B0C10111579
:1062960000160A1322312900000000AA2E192B37F6
:0862A6002E712E512E9A2E00DC
:107E00000F92CDB7DEB7112484B714BE81FFF1D035
:107E100082E08093C00088E18093C10086E0809377
:107E2000C20080E18093C4008EE0CDD088249924E4
:107E3000CC24C394F5E0DF2EE1E1EE2E73E0F72EC3
:107E4000B6D0082F813479F4B2D08983C2D0898129
:107E5000823811F481E005C0813811F485E001C059
:107E600083E09ED09AC0823411F484E103C085344B
:107E700019F485E0B6D091C0853561F498D0082F0B
:107E800010E095D090E0982E8824802A912A880CC2
:107E9000991C82C0863521F484E0A3D080E0E1CF34
:107EA000843609F04CC083D082D0A82E80D0B82E62
:107EB00000E011E07CD0F80181938F01AE16D1F77C
:107EC00088D0FB2DF53489F4E0E0F1E00BC0F9999E
:107ED000FECF92BC81BC0894811C911C819180BD15
:107EE000FA9AF99AEA1598F358C08B2D863409F05E
:107EF00054C0F401F7BEE89507B600FCFDCFF401CD
:107F0000A0E0B1E02C9130E011968C91119790E0B7
:107F1000982F8827822B932B12960C01C7BEE895C9
:107F20001124329681E0A038B80761F7F401D7BE7A
:107F3000E89507B600FCFDCFE7BEE8952EC0843774
:107F4000F1F435D034D0182F32D0B82E42D0FB2DDA
:107F5000F63421F4F40105914F010CC0FB2DF534EA
:107F600049F4F999FECF92BC81BC0894811C911C04
:107F7000F89A00B5802F14D0115049F70EC08537FC
:107F800039F427D08EE10CD085E90AD08FE069CF93
:107F9000813511F488E017D01CD080E101D050CF9A
:107FA0009091C00095FFFCCF8093C600089580910A
:107FB000C00087FFFCCF8091C00084FD01C0A89560
:107FC0008091C6000895E0E6F0E098E19083808318
:107FD0000895EDDF803219F088E0F5DFFFCF84E10E
:107FE000DFCF1F93182FE3DF1150E9F7F2DF1F9166
:0E7FF0000895282E80E0E7DFEE27FF27099492
:027FFE0001057B
:0400000300007E007B
:00000001FF
